:1000000000308A0004280000FF238316900000308F
:100010008A00882830308400000803191D28013028
:10002000A100A001A00B1228A10B11284A30A000AA
:10003000A00B18281B28800B0F280800831685109A
:1000400083128510831605108312051083168515FB
:1000500085128312851683160512831205128316E4
:10006000051583129C28A401A501A601A7019830BB
:10007000A8008830A9007F30AA009D280512013011
:10008000B0000A2005160A30B0000A209E28B308E6
:1000900003194C2805144D28051000008514000094
:1000A000851008008512B3014720B30147200130B5
:1000B000B3004720B3014720B3014720B3014720D5
:1000C000B3014720B3014720B2013208073C031CAB
:1000D0007528B01F6F280130B30047207128B30185
:1000E00047200310B00DB20A6528B2013208073C60
:1000F000031C8628B11F80280130B30047208228C6
:10010000B30147200310B10DB20A76288516080006
:1001100084011F3083051F1383161F109F101F11AA
:100120009F11073083129900FF3083168500C83075
:100130008312B0000A201E2833283E28B00124086C
:10014000B10052200130B0002508B1005220023029
:10015000B0002608B10052200330B0002708B100DB
:1001600052200430B0002808B10052200530B00001
:100170002908B10052200630B0002A08B1005220F0
:10018000051DC5289830AE00C7289030AE0028085D
:100190002E020319D2282E08A8000430B000280827
:0801A000B1005220C0286300E9
:02400E00043F6D
:00000001FF
